:0200000480007A
:100000006F00C004732F2034930F8000630AFF0336
:10001000930F90006306FF03930FB0006302FF038A
:10002000170F0000130F0F1363040F0067000F007A
:10003000732F203463540F006F00400093E19153FD
:10004000171F000023203FFC6FF09FFF732540F136
:1000500063100500970200009382020173905230F2
:10006000735000189702000093820202739052307E
:10007000B70200809382F2FF7390023B9302F0017B
:100080007390023A9702000093828201739052307B
:100090007350203073503030735040309301000063
:1000A00097020000938242F67390523013051000BD
:1000B0001315F501634C05000F00F00F93011000BC
:1000C0009308D005130500007300000093020000A0
:1000D000638E020073905210B7B2000093829210A8
:1000E0007390223073232030E39A62F4735000300F
:1000F00037250000130505807320053097020000A6
:100100009382420173901234732540F173002030C2
:1001100093012000730010006F0080006310300214
:100120000F00F00F638001009391110093E1110023
:100130009308D00513850100730000000F00F00F35
:10014000930110009308D005130500007300000010
:1001500013033000F3222034E39462FC1703000001
:10016000130383FBF3221034E39C62FA6FF01FFD4C
:10017000731000C00000000000000000000000003C
:1010000000000000000000000000000000000000E0
:1010100000000000000000000000000000000000D0
:1010200000000000000000000000000000000000C0
:1010300000000000000000000000000000000000B0
:081040000000000000000000A8
:040000058000000077
:00000001FF
